:10000000DDC1F6C1F5C1F4C1F3C1F2C1F1C1F0C166
:10001000EFC10AC7EDC1CEC5F2C5EAC18CC6E8C1C1
:10002000E7C1E6C1E5C13078004D6F7665206469AF
:10003000616C20746F20313030306D414800507257
:10004000657373203C4E3E20746F20636F6E74693D
:100050006E7565004D6F7665206469616C20746F04
:1000600020333030306D4148005072657373203C4E
:100070004E3E20746F20636F6E74696E7565004923
:100080006E73657274206120736574206F662063DF
:10009000656C6C73207769746820616E20416D6DAA
:1000A0006574657220696E2073657269657320617D
:1000B0006E642061646A757374207468652063756A
:1000C0007272656E7420746F203130306D41005053
:1000D00072657373203C553E20746F20696E6372A5
:1000E00065616365207468652063757272656E74FE
:1000F00020616E64203C443E20746F20646563720E
:10010000656163652069742E005768656E207468A8
:10011000652063757272656E742069732066696EFE
:10012000616C6C79207365742C2070726573732018
:100130003C4E3E00496E7365727420612073657495
:10014000206F662063656C6C73207769746820612A
:100150006E20416D6D6574657220696E20736572E5
:1001600069657320616E642061646A7573742074BC
:1001700068652063757272656E7420746F20333009
:10018000306D41005072657373203C553E20746F92
:1001900020696E63726561636520746865206375AC
:1001A0007272656E7420616E64203C443E20746FF0
:1001B0002064656372656163652069742E00576809
:1001C000656E207468652063757272656E7420694F
:1001D000732066696E616C6C79207365742C207075
:1001E00072657373203C4E3E002D2D2D2D2D2D2D2F
:1001F0002D2D2D2D2D2D2D2D2D2D2D2D2D2D2D2D2F
:100200002D2D2D2D2D00506F74206C6F636174693E
:100210006F6E20666F72203130306D41203D2000BE
:100220002000536574706F696E7420666F722031A0
:1002300030306D41203D20002000506F74206C6FE5
:10024000636174696F6E20666F72203330306D4168
:10025000203D20002000536574706F696E74206625
:100260006F72203330306D41203D20002D2D2D2D1B
:100270002D2D2D2D2D2D2D2D2D2D2D2D2D2D2D2DAE
:100280002D2D2D2D2D2D2D2D0020002000506F7493
:10029000206C696E65617269747920636865636B4F
:1002A000004D6F76652074686520504F5420616E54
:1002B0006420636865636B2074686520637572727F
:1002C000656E74206F6E20746865206D657465724C
:1002D000005072657373203C4E3E20746F20636F34
:1002E0006E74696E75650066726F6D207777772E14
:1002F0006F70656E642E636F2E7A610050574D20CB
:100300006E696D6820636861726765720046572088
:1003100076657273696F6E20302E310048572076F3
:10032000657273696F6E20312E30005479706520CC
:100330003C7365743E20746F2063616C6962726106
:100340007465207468652073656C6563746F7200F2
:1003500054696D6520666F722063616C69627261B9
:1003600074696F6E206973206F7665722100576122
:100370006974696E6720666F72206361706163697A
:10038000747920656E747279004361706163697479
:1003900079207365742C206368617267696E6720C9
:1003A00073746172746564004368617267696E6733
:1003B00020636F6D706C65746564000011241FBE4E
:1003C000CFE5D4E0DEBFCDBF10E0A0E6B0E0E2E6CE
:1003D000FFE002C005900D92A236B107D9F710E0F8
:1003E000A2E6B0E001C01D92AF3DB107E1F7D6C271
:1003F00007CECF92DF92EF92FF920F931F93CF938E
:10040000DF9381E0CED4DBD4DAD4D9D4E0906D0090
:10041000F0906E002091730030917400C0907100D4
:10042000D090720000916F00109170008E159F05A2
:10043000E0F08E199F09EC01EE27FF272C193D09EA
:1004400044275527BE01CF0137D50E191F09980142
:100450004427552750D5FA01E901C601AA27BB2731
:10046000C80FD91FEA1FFB1F1CC0A701481B590B4F
:10047000EA01EE27FF272C193D0944275527BE0125
:10048000CF011AD50E191F0998014427552733D5D6
:10049000C601AA27BB27821B930BA40BB50BFD013A
:1004A000EC01D0936300C093620080E07AD487D4DB
:1004B00086D4DF91CF911F910F91FF90EF90DF9045
:1004C000CF9008951F93CF93DF93EC0186E290E0E5
:1004D00010D413E0CE01892F992782958F708F70E9
:1004E0008A3010F4805D01C0895CDAD384E0CC0FDF
:1004F000DD1F8A95E1F7115017FFECCFDF91CF9107
:100500001F9108950F931F93CF93DF9371D4882386
:1005100009F4BCC054D4AA27BB27209164003091B1
:1005200065004091660050916700280F391F4A1FEF
:100530005B1F2093640030936500409366005093E6
:10054000670080916800803110F0109268008091FF
:1005500068008F5F80936800813009F097C0DA01EE
:10056000C90173E0B695A795979587957A95D1F7C8
:100570008093640090936500A0936600B093670039
:100580008093690090936A00A0936B00B0936C0015
:100590000091620010916300E801EE27FF278C179D
:1005A0009D07AE07BF0738F560916000643618F507
:1005B0009C01AD01762F7F5FDA01C90163E0B6953A
:1005C000A795979587956A95D1F7280F391F4A1FE8
:1005D0005B1F2C173D074E075F0718F4672F743613
:1005E00048F32093690030936A0040936B00509366
:1005F0006C00709360008091640090916500A09100
:100600006600B09167008093690090936A00A093A0
:100610006B00B0936C00E801EE27FF27C817D907DD
:10062000EA07FB0738F560916000653018F19C011E
:10063000AD01762F7150DA01C90163E0B695A79537
:10064000979587956A95D1F7281B390B4A0B5B0B59
:10065000C217D307E407F50718F4672F753048F77A
:100660002093690030936A0040936B0050936C00B4
:100670007093600080916000992775D21092640099
:10068000109265001092660010926700DF91CF9182
:100690001F910F910895FF920F931F93CF93DF93B4
:1006A00010E0F12E012FC12F80ED97E0A0E0B0E027
:1006B0008093DB009093DC00A093DD00B093DE001C
:1006C0008091DB009091DC00A091DD00B091DE0014
:1006D0000097A105B10509F43FC18AD381116FD3F9
:1006E000F1D2882389F080ED97E0A0E0B0E080931C
:1006F000DB009093DC00A093DD00B093DE00F12ED0
:10070000102FBCD2082FCF5F8091DB009091DC00CE
:10071000A091DD00B091DE000097A105B10511F0B8
:10072000C330D8F2C33009F017C183E7F81609F0D7
:1007300013C1153609F010C1043709F00DC181E06D
:1007400030D33DD33CD389E290E0E4D28EE390E015
:10075000E1D208C04DD3882329F031D390936E00A5
:1007600080936D00AFD28823A9F388D28E3659F7D3
:1007700084E590E0CFD289E690E0CCD208C038D3AF
:10078000882329F01CD39093700080936F009AD235
:100790008823A9F373D28E3659F780E002D30FD3A2
:1007A0000ED310E08CEC90E0909363008093620095
:1007B0008FE790E0AFD28FEC90E0ACD289E091E08F
:1007C000A9D280D28823C9F059D2182F843641F497
:1007D0008091620090916300009779F0019709C0C1
:1007E000853759F4809162009091630097FD05C0B0
:1007F0000196909363008093620084DE1E3609F7B1
:1008000080916200909163009093720080937100D8
:1008100010E088E693E0909363008093620084E3A5
:1008200091E078D284E891E075D28EEB91E072D2BB
:1008300049D28823C9F022D2182F843641F48091FE
:10084000620090916300009779F0019709C08537A5
:1008500059F4809162009091630097FD05C0019664
:1008600090936300809362004DDE1E3609F78091FD
:1008700062009091630090937400809373001092D3
:1008800063001092620089EE91E044D286E092E02B
:1008900030D280916D0090916E0014DE80E292E083
:1008A00039D282E292E025D280917100909172005B
:1008B00009DE88E392E02ED28AE392E01AD2809198
:1008C0006F0090917000FEDD84E592E023D286E512
:1008D00092E00FD28091730090917400F3DD8CE66A
:1008E00092E018D289E892E015D28BE892E012D219
:1008F00010E08DE892E00ED281EA92E00BD281ED19
:1009000092E008D2DFD1882311F0B8D1182F71DD21
:10091000CFE0D7E2F7DD2197D7FFFCCF1E3691F766
:1009200060E070E080916D0090916E00A6D262E070
:1009300070E080916F00909170009FD264E070E051
:10094000809171009091720098D266E070E0809181
:1009500073009091740091D280E090E09CD29093CB
:100960006E0080936D0082E090E095D290937000CD
:1009700080936F0084E090E08ED290937200809319
:10098000710086E090E087D29093740080937300AA
:10099000DF91CF911F910F91FF900895CFE5D4E0A3
:1009A000DEBFCDBF80EC81BB12BA88E085BB66E0BC
:1009B0008FEC90E0DED0CCD080E0F3D130D27894D0
:1009C00087EE92E0A7D18CEF92E0A4D18DE093E086
:1009D000A1D18CE193E09ED18BE293E09BD1369A3A
:1009E00080E482BB58DE1092DB001092DC00109293
:1009F000DD001092DE0012BA80E593E08BD18EE626
:100A000093E088D180E090E0AED01092DB001092AD
:100A1000DC001092DD001092DE009B9B31C0E8D11B
:100A20008111CDD14FD1811110D1E3DC8091DB0058
:100A30009091DC00A091DD00B091DE000097A1054F
:100A4000B10561F488EE91E0A0E0B0E08093DB00B6
:100A50009093DC00A093DD00B093DE008091DB007A
:100A60009091DC00A091DD00B091DE00C397A1055C
:100A7000B10510F012BA02C080E482BB9B99CFCFBF
:100A800089E893E036D18EEB94E0AFEEB2E080934C
:100A9000DB009093DC00A093DD00B093DE0080913A
:100AA000DB009091DC00A091DD00B091DE000097AA
:100AB000A105B10581F026DD8091DB009091DC007D
:100AC000A091DD00B091DE0091FD02C080E401C084
:100AD00080E882BBE4CF88EA93E00BD180E090E02D
:100AE00042D01092DB001092DC001092DD001092D8
:100AF000DE007ED1811163D1E5D08111A6D0809135
:100B0000DB009091DC00A091DD00B091DE00009749
:100B1000A105B10561F488EC90E0A0E0B0E080931D
:100B2000DB009093DC00A093DD00B093DE008091A9
:100B3000DB009091DC00A091DD00B091DE00C39756
:100B4000A105B10510F012BAD4CF80E882BBD1CF95
:100B50008AE88FBD81E18EBDB99AC1988FE790E098
:100B600097BD86BD08959C01832F99278BBD2ABD13
:100B700008959C0188E02030380740F02F5F3F4FF8
:100B800036952795215030401BB802C082E08BB9C2
:100B9000832F99278F7080BD29B988E98AB9606849
:100BA00060BD10929600109295001092B8001092BD
:100BB000B70008951F920F920FB60F9211242F9332
:100BC0008F939F93EF93FF932CB1E0919500EF5F8C
:100BD0009E2F9F71E15080919600981731F0FF276A
:100BE000EB58FF4F208390939500FF91EF919F91D9
:100BF0008F912F910F900FBE0F901F9018951F92FD
:100C00000F920FB60F9211248F939F93EF93FF9340
:100C10009091B7008091B800981769F08091B80062
:100C20008F5F8F718093B800E82FFF27E956FF4F41
:100C300080818CB901C05598FF91EF919F918F9160
:100C40000F900FBE0F901F901895209196009091D5
:100C50009500809195009817D1F7809195008217A3
:100C6000A1F3E22FFF27EB58FF4F9081822F8F5F78
:100C70008F7180939600892F99270895E6DF982F2A
:100C800081548A3108F4905E892F99270895DDDF19
:100C9000982F81568A3108F49052892F9927089508
:100CA000282F9091B7009F5F9F718091B80098178F
:100CB000E1F3E92FFF27E956FF4F20839093B70018
:100CC000559A089530E0209195009091960080917A
:100CD0009500281331E080919600981799F73323F7
:100CE00089F7291719F480E090E0089581E090E0F9
:100CF0000895CF93DF93EC01FC0121968491882322
:100D000031F0CEDFFE01219684918823D1F7DF9167
:100D1000CF910895CF93DF93EC01FE01219684914A
:100D2000882311F0BDDFF9CF8DE0BADF8AE0B8DFAC
:100D3000DF91CF9108951F920F920FB60F92112459
:100D40002F934F935F938F939F93EF93FF9324B1D0
:100D500085B19927582F4427420F511DE091D900A2
:100D60009091DA008091DA009817D1F7EF5F8E2F1B
:100D70008F70E150891749F0FF27EE0FFF1FE754EE
:100D8000FF4F518340838093D900FF91EF919F9152
:100D90008F915F914F912F910F900FBE0F901F90E9
:100DA00018951092DA001092DA001092D900109281
:100DB000D9009FEB96B98F70806C87B90895909198
:100DC000DA002091D9008091D9002817D1F7921725
:100DD000B1F3E92FFF27EE0FFF1FE754FF4F2081EC
:100DE0003181892F8F5F8F708093DA00C901089558
:100DF00030E02091D9009091DA008091D900281339
:100E000031E08091DA00981799F7332389F7291791
:100E100019F480E090E0089581E090E0089583E087
:100E200083BF81E089BF08951F920F920FB60F9282
:100E300011248F939F93AF93BF938091DB00909188
:100E4000DC00A091DD00B091DE000097A105B105A6
:100E500059F00197A109B1098093DB009093DC0060
:100E6000A093DD00B093DE00BF91AF919F918F9171
:100E70000F900FBE0F901F9018959B01E199FECF28
:100E8000D9012F5F3F4F082E60D0E199FECFD901E5
:100E9000092E5BD008959C01E199FECFD9012F5F07
:100EA0003F4F4BD0802D482FE199FECFD90145D03F
:100EB000802D582FCA010895629FD001739FF001C1
:100EC000829FE00DF11D649FE00DF11D929FF00DDA
:100ED000839FF00D749FF00D659FF00D9927729F11
:100EE000B00DE11DF91F639FB00DE11DF91FBD019C
:100EF000CF0111240895A1E21A2EAA1BBB1BFD01EC
:100F00000DC0AA1FBB1FEE1FFF1FA217B307E407E8
:100F1000F50720F0A21BB30BE40BF50B661F771F40
:100F2000881F991F1A9469F7609570958095909520
:100F30009B01AC01BD01CF010895E199FECFBFBB7C
:100F4000AEBBE09A11960DB20895E199FECFBFBBFA
:100F5000AEBB0DBA11960FB6F894E29AE19A0FBEA5
:020F60000895F2
:020F6200040089
:00000001FF
